:0CFD0300011200010C00010B00010E00B9
:10FC2C0012F90C12FD5712FDD1E50CB4FF14E519B5
:10FC3C00D39400400DD5190AE47834F67F0AFE12ED
:10FC4C00FDB47838E6600712FC69E47838F620B029
:0DFC5C00087838E6700312FA1E050C80C906
:10F90C00C2087580FF43BF027B007A0079087F0034
:10F91C007EEE12FDA8AD08E4FFFE12FD9B7B007A83
:10F92C000079097F017EEE12FDA8AD097F017E00F2
:10F93C0012FD9B7B007A0079137F027EEE12FDA8EC
:10F94C00AD137F027E0012FD9B7B007A0079147F41
:10F95C00037EEE12FDA8AD147F037E0012FD9B7B8F
:10F96C00007A0079117F047EEE12FDA8AD117F04A0
:10F97C007E0012FD9B7B007A00790F7F057EEE12D4
:10F98C00FDA8AD0F7F057E0012FD9B7B007A0079F0
:10F99C001B7F067EEE12FDA8AD1B7F067E0012FDBE
:10F9AC009B7B007A0079157F077EEE12FDA8AD15C2
:10F9BC007F077E0012FD9B7B007A00790A7F087E10
:10F9CC00EE12FDA8AD0A7F087E0012FD9B7B007A2B
:10F9DC0000790D7F097EEE12FDA8AD0D7F097E002A
:10F9EC0012FD9B7D207F0B7E0012FD9B7B007A001D
:10F9FC0079107F107EEE12FDA8AD107F107E0012E4
:10FA0C00FD9BE5D85408FFE5107006BF0803020201
:02FA1C000022C6
:04FDD100759FA72251
:0BFDB400EF1FAC0670011E4C70F62221
:10F28C0000C1814001C0804101C0804100C181406A
:10F29C0001C0804100C1814000C1814001C080415A
:10F2AC0001C0804100C1814000C1814001C080414A
:10F2BC0000C1814001C0804101C0804100C181403A
:10F2CC0001C0804100C1814000C1814001C080412A
:10F2DC0000C1814001C0804101C0804100C181401A
:10F2EC0000C1814001C0804101C0804100C181400A
:10F2FC0001C0804100C1814000C1814001C08041FA
:10F30C0001C0804100C1814000C1814001C08041E9
:10F31C0000C1814001C0804101C0804100C18140D9
:10F32C0000C1814001C0804101C0804100C18140C9
:10F33C0001C0804100C1814000C1814001C08041B9
:10F34C0000C1814001C0804101C0804100C18140A9
:10F35C0001C0804100C1814000C1814001C0804199
:10F36C0001C0804100C1814000C1814001C0804189
:10F37C0000C1814001C0804101C0804100C1814079
:10F38C0000C0C101C30302C2C60607C705C5C40439
:10F39C00CC0C0DCD0FCFCE0E0ACACB0BC90908C8A9
:10F3AC00D81819D91BDBDA1A1EDEDF1FDD1D1CDC99
:10F3BC0014D4D515D71716D6D21213D311D1D01009
:10F3CC00F03031F133F3F23236F6F737F53534F4F9
:10F3DC003CFCFD3DFF3F3EFEFA3A3BFB39F9F83869
:10F3EC0028E8E929EB2B2AEAEE2E2FEF2DEDEC2C59
:10F3FC00E42425E527E7E62622E2E323E12120E0C9
:10F40C00A06061A163A3A26266A6A767A56564A4B8
:10F41C006CACAD6DAF6F6EAEAA6A6BAB69A9A86828
:10F42C0078B8B979BB7B7ABABE7E7FBF7DBDBC7C18
:10F43C00B47475B577B7B67672B2B373B17170B088
:10F44C005090915193535292965657975595945478
:10F45C009C5C5D9D5F9F9E5E5A9A9B5B99595898E8
:10F46C00884849894B8B8A4A4E8E8F4F8D4D4C8CD8
:10F47C004484854587474686824243834181804048
:10FD0F000116FF011D010134000117960139000191
:05FD1F003500011B008E
:10FD5700C2B2E47834F67838F6E51B6003B4FF03E3
:04FD6700751BFE22E8
:0DFD8E00C2B2E47834F67838F67517962284
:09FDBF00D2B27F0A7E0002FDB4FD
:10FA1E00E4F520D2087F04FE12FDB4C208A2B09213
:10FA2E0000D2087F037E0012FDB4C208A2B092017C
:10FA3E00D2087F037E0012FDB4C208A2B09202D299
:10FA4E00087F037E0012FDB4C208A2B09203D20852
:10FA5E007F037E0012FDB4C208A2B09204D2087FCA
:10FA6E00037E0012FDB4C208A2B09205D2087F0335
:10FA7E007E0012FDB4C208A2B09206D2087F037EA9
:10FA8E000012FDB4C208A2B09207D2087834E6C3C1
:10FA9E0094965007E606243AF8A620C2087834E673
:10FAAE00FFB517057838760122EF64077020783B92
:10FABE00E6FE64036004EEB4060475170822EEB485
:10FACE0010087840E62409F5172275179622EFB430
:10FADE0001047519C822EFB40309783BE6B4190383
:04FAEE007517062260
:10FCD9007833E6FF7E15D208C2B1DEFEE4FDEF13EC
:10FCE90092B1EFC313FF7E12DEFE0DBD08F0D2B153
:0AFCF9007F087E0012FDB4C208224D
:10FC690012F7D4501312FDBF12FDC812F48C5005BF
:10FC790012F661800302FD8E12FD8EE516B401179E
:10FC8900E4FD7F107EEE12FCA1AD1B7F067EEF1214
:08FC9900FCA1759F8080FE2292
:10F7D4007834E665176002C322783AE6FFF4600ADB
:10F7E400EF651B6005EF6002C322783BE664197085
:10F7F4007AFB7A00793A7D0412FBA88E228F237853
:10F804003EE6FE08E67C002400FFEC3EFEEF6523A6
:10F814007003EE65226002C322783DE6FF18E6FE1F
:10F82400C39F4004AD078002AD06EEC39F4004AF02
:10F83400068000E51BC39D4006E51BD39F4002C321
:10F8440022AF0C7E0012FC2212FBEB7C007D1E1208
:10F85400FB1D8D25E4F524E524C39525500B7F6419
:10F864007E0012FDB4052480EED322783BE6FF64CB
:10F8740003600CEF64066007EF64106002C3227833
:10F884003CE6FE08E67C002400FFEC3EFEEF640A42
:10F894004E7042783BE6B4030C12FBEB7C007D0512
:10F8A40012FB1D8D1CE51C64016002C322AF0C7E9B
:10F8B4000012FC2212FBEB7C007D1412FB1D8D2533
:10F8C400E4F524E524C39525500B7F647E0012FDE6
:10F8D400B4052480EE7B007A00793AE51724FEFD16
:10F8E40012FBA88E228F2374382517F8E6FE74398C
:0AF8F4002517F8E67C002400FFEC65
:0EF8FE003EFEEFB52306EEB52202D322C32252
:10F66100E4F525783BE6B4061AE4F525743A252538
:10F67100F8E6FF12FCDD12FDD10525E525C394084E
:10F6810040EA22783BE66403600302F76708E6FE7E
:10F6910008E67C002400F523EC3EF522783FE6F5F0
:10F6A10024783AE6FF12FCDD783AE6FF12FD417854
:10F6B1003BE6FF12FCDD783BE6FF12FD41E5242528
:10F6C100E0FF12FCDDE52425E0FF12FD41E525C345
:10F6D1009524400302F75AE4FF12FCDDE4FF12FD1A
:10F6E10041E51DB47B167E00E5232525FFEE35227D
:10F6F100FE7B007A00792612FDA8804E7E00E5236C
:10F701002525FFEE3522FEC3EF940CEE9400500B3D
:10F711007B007A00792612FD6B802F7E00E5232580
:10F7210025FFEE3522FEEF64204E700585BF268051
:10F7310019EF642D4E7005851D26800EEF64304E45
:10F7410070058518268003752601AF2612FCDDAFF2
:10F751002612FD41052502F6CE12FCD97836E6FFC8
:10F7610012FCDD02FDD1783BE66410702CF52574A6
:10F771003A2525F8E6FF12FCDD743A2525F8E6FF67
:10F7810012FD410525E525C3940640E312FCD97815
:10F7910036E6FF12FCDD02FDD1783BE664197032DA
:03F7A10018E6FF68
:10F7A40012FCDD783AE6FF12FD41783BE6FF12FCDD
:10F7B400DD783BE6FF12FD41AF1B12FCDDAF1B12EF
:10F7C400FD4112FCD97836E6FF12FCDD12FDD12290
:10F48C00783BE664067064783DE6FFB406117E00B6
:10F49C00783FE6FD12FD9B783FE6F51B02F5F07810
:10F4AC003DE6B40A1CE51C6401600302F5F0783FEC
:10F4BC00E6FD7F067E0012FD9B783FE6F51B02F50C
:10F4CC00F0783DE6FFB410117E00783FE6FD12FDAA
:10F4DC009B783FE6F51602F5F0783DE6642D600367
:10F4EC0002F5F0783FE6F51D02F5F0783BE6641086
:10F4FC00600302F5F0783FE6F52A08E6FD783CE675
:10F50C00FCFE08E6F97A002400F525EA3EF5248C89
:10F51C00288929E52A6D7036F526F527C3E5279548
:10F52C002AE5269400506074412527F8E6F523E57A
:10F53C00252527FFE5243526FEAD2312FCA140012D
:10F54C002212FDD10527E52770D2052680CEE4F5E1
:10F55C0026F527C3E527952AE52694005029E527AB
:10F56C0025E02442F8E6F523E5252527FFE524359B
:10F57C0026FEAD2312FCA140012212FDD10527E588
:10F58C002770D0052680CC783906E664087055784B
:10F59C0035E675F002A42411FFE5F034EEFEE4FD2F
:10F5AC0012FCA17835E675F002A42412FFE5F034C4
:0FF5BC00EEFEE4FD12FCA1783506E675F002A420
:10F5CB002411FFE5F034EEFEAD2812FCA17835E6F0
:10F5DB0075F002A42412FFE5F034EEFEAD2912FC07
:10F5EB00A1E47839F6E516B47F0CE47839F6783572
:10F5FB00F675167E805EE516B43F19E4F522AF2250
:10F60B0012FD2912FDD10522E522C3946440EF754A
:10F61B00163E8040E516B4330B12FDD112FD7E75FC
:10F62B0016348030E516B41F2312FDD17D1F7F10D9
:10F63B007EEE12FCA17DF07F117EEE12FCA17DF01F
:10F64B007F127EEE12FCA175161E8008E516B40122
:06F65B000312FDD1D322D1
:09FDC800783676FF783376FF22CD
:10FD41007833E66FFF90F28C937836667933F7EF6C
:06FD510090F38C93F622F2
:10FBA8008B268A2789288D29752A00752BFF7DFFCA
:10FBB800AF291529EF6026AB260528E528AA277066
:10FBC80002052714F912FAF2652BFF90F28C936D57
:10FBD800752A00F52BEF90F38C93FD80D3E52BFE6F
:03FBE800EDFF220C
:04FD2400410000009A
:06FCA1008E2B8F2C8D2D2F
:10FCA70012FDD175F65575F6AA75F65575BF04851B
:10FCB7002DF6E52BF5F4852CF575F7807B007A009A
:10FCC700792EAF2CAE2B12FDA8E52EB52D02D3222F
:01FCD700C369
:01FCD8002209
:10FD290075F65575F6AA75F65575BF04EF25E0F514
:08FD3900F4E4F5F575F78222F0
:10FD7E0075F65575F6AA75F65575BF0475F7832297
:0BFDA8008F828E83E49312FB0B7F011F
:01FDB300222D
:0DFD9B0074002FF582E43400F583EDF022B2
:10FD6B0074002FF582E43400F583E012FB0B12FADA
:03FD7B00F2FF2272
:01F0000020EF
:0300000002F20009
:0CF20000787FE4F6D8FD7581CF02F2475C
:10FAF200BB010689828A83E0225002E722BBFE0212
:09FB0200E32289828A83E4932244
:10FB0B00BB010689828A83F0225002F722BBFE01D9
:02FB1B00F322D3
:10FB1D00C2D5EC30E709B2D5E4C39DFDE49CFCEE03
:10FB2D0030E715B2D5E4C39FFFE49EFE12FB53C32D
:10FB3D00E49DFDE49CFC800312FB5330D507C3E428
:06FB4D009FFFE49EFE2272
:10FBEB00AC2FAD30AE31AF32780FEFA2E2EC20E6A6
:10FBFB0001B35D5E5FF47004FCFDFEFFEF13FFEEDF
:10FC0B0013FEED13FDEC13FCD8E08C2F8D308E31F1
:10FC1B008F32EE547FFE228E2F8F30E4F531F5328A
:01FC2B0022B6
:10F20C0002FC2CE493A3F8E493A34003F68001F2F0
:10F21C0008DFF48029E493A3F85407240CC8C33303
:10F22C00C4540F4420C8834004F456800146F6DFD2
:10F23C00E4800B010204081020408090FD03E47E62
:10F24C00019360BCA3FF543F30E509541FFEE493C7
:10F25C00A360010ECF54C025E060A840B8E493A38E
:10F26C00FAE493A3F8E493A3C8C582C8CAC583CAB9
:10F27C00F0A3C8C582C8CAC583CADFE9DEE780BE71
:01FD280000DA
:10FB5300BC000BBE0029EF8DF084FFADF022E4CC96
:10FB6300F875F008EF2FFFEE33FEEC33FCEE9DEC5F
:10FB7300984005FCEE9DFE0FD5F0E9E4CEFD22EDA5
:10FB8300F8F5F0EE8420D21CFEADF075F008EF2FEF
:10FB9300FFED33FD4007985006D5F0F222C398FDE0
:05FBA3000FD5F0EA227D
:00000001FF
